:020000040000FA
:1000000083160030860083124F20112052200A20D0
:100010008D0A05286F3C03190E2808004F2005287B
:10002000080009300D020319392808300D020319A0
:100030003B2807300D0203193D2806300D02031935
:100040003F2805300D020319412804300D02031921
:10005000432803300D020319452802300D0203190D
:10006000472801300D020319492800300D020319F9
:100070004B286F304D287F304D2807304D287D307C
:100080004D286D304D2866304D284F304D285B305F
:100090004D2806304D283F304D288600080000309E
:1000A0008D00080083160430810083120630810021
:1000B0007D308C000108031D5A28063081008C0B0E
:0400C0005A280800B2
:02400E00F13F80
:00000001FF
